:100000000C94D1060C9418070C9418070C9418073C
:100010000C9418070C9418070C9418070C941807E4
:100020000C9418070C9418070C948E2B0C94602CCD
:100030000C94B41D0C9418070C9418070C94180712
:100040000C9418070C9418070C9418070C941807B4
:100050000C9418070C94281E0C9418070C9418077D
:100060000C9418070C9418070C9418070C94180794
:100070000C9418070C9418070C9418070C94180784
:100080000C9418070C9418070C9418070C94180774
:100090000C9418070C9418070C9418070C94180764
:1000A0000C9418070C9418070C94180706090809F3
:1000B00013090A090C090E09100912091509170973
:1000C000190924091B091D091F09210923092609EA
:1000D00096139613C813C813061426148A158A1586
:1000E00068148A15091509157A158A158A15831554
:1000F00016151615161516151615161516151615A8
:100100001615161516151615161516151615161597
:10011000271535153C1543154D15191619162B16AF
:100120002B1622162B162B162B16191619162716F8
:100130002B162B162716CD2CF42CE62DF42CE62DA1
:10014000402D632DE62DB92DC82D29001E001F005E
:100150002000210022002300240025002600270083
:100160002D002E00350031002B0014001A0008006D
:10017000150017001C0018000C00120013002F00BF
:1001800030002A004B00E0000400160007000900C0
:100190000A000B000D000E000F0033003400280091
:1001A00000004E00E1001D001B00060019000500C4
:1001B00011001000360037003800E5000000520042
:1001C0000251E0000000005700002C000151000027
:1001D0002C000000015700000000500051004F00AB
:1001E0000100010001000100010001000100010007
:1001F00001000100010001000100010001003900BF
:10020000010001000100010001000100460047005B
:1002100048000100010001004C00010001003A000B
:100220003B003C003D003E003F000100010001009A
:100230000100010001000000010001004000410038
:100240004200430044004500010001000100650038
:100250000100000001000100010000000100000099
:10026000010001000000010000000100000000008A
:100270000100010001000100010001000100010076
:100280000100010001000100010001000100010066
:10029000010001003900010001000100010001001E
:1002A00001000100010001000100010001004C00FB
:1002B0004A000100010001000100010001000100ED
:1002C00001000100010001000100AE0000004D002E
:1002D00001000100010001000100005C01000100BB
:1002E00001000100010001000000A900010001005F
:1002F00000000100000001000100000001000000FA
:10030000010000000000AC00AA00AB0044454255CB
:10031000473A2064697361626C65642E0A00444543
:100320004255473A20656E61626C65642E0A000A88
:10033000002530313662003A200025303258000A5C
:10034000722F6320303132333435363738394142F9
:10035000434445460A000A002530325820006B65A8
:1003600079626F6172645F7265706F72743A2000B7
:100370000A0025303258006B6579626F6172645FE4
:100380007365745F6C65643A2000290A0025750066
:100390002F002575005D28002564002000256400DD
:1003A000200025640020002564007C0025303258A0
:1003B000006D6F7573656B6579205B62746E7C7818
:1003C0002079207620685D287265702F61636C2922
:1003D0003A205B006D6B5F776865656C5F74696D73
:1003E000655F746F5F6D6178203D2025640A006D44
:1003F0006B5F776865656C5F6D61785F737065656D
:1004000064203D2025640A006D6B5F74696D655F33
:10041000746F5F6D6178203D2025640A006D6B5F0D
:100420006D61785F7370656564203D2025640A0006
:100430006D6B5F696E74657276616C203D2025641A
:100440000A006D6B5F64656C6179203D2025640A4C
:10045000006D6B5F776865656C5F74696D655F746F
:100460006F5F6D6178203D2025640A006D6B5F77BA
:100470006865656C5F6D61785F7370656564203D6C
:100480002025640A006D6B5F74696D655F746F5F32
:100490006D6178203D2025640A006D6B5F6D617889
:1004A0005F7370656564203D2025640A006D6B5F95
:1004B000696E74657276616C203D2025640A006D5A
:1004C0006B5F64656C6179203D2025640A000A0039
:1004D000257500363A20776865656C5F74696D65CF
:1004E0005F746F5F6D61783A20000A0025750035F2
:1004F0003A20776865656C5F6D61785F73706565DC
:10050000643A20000A00257500343A2074696D654C
:100510005F746F5F6D61783A20000A0025750033C3
:100520003A206D61785F73706565643A20000A0057
:10053000257500323A20696E74657276616C286D9B
:1005400073293A20000A00257500313A2064656C51
:100550006179282A31306D73293A20000A092D204B
:1005600056616C756573202D0A004D3E004D256463
:100570003E20003F007365742064656661756C748D
:100580000A00433E200077686572652064656C74DC
:10059000613A20637572736F723D25642C20776811
:1005A00065656C3D25640A53656520687474703A0E
:1005B0002F2F656E2E77696B6970656469612E6F88
:1005C00072672F77696B692F4D6F7573655F6B6508
:1005D00079730A000A092D204D6F7573656B657973
:1005E000202D0A4553432F713A09717569740A31F8
:1005F0003A0964656C6179282A31306D73290A32B1
:100600003A09696E74657276616C286D73290A33D4
:100610003A096D61785F73706565640A343A0974EC
:10062000696D655F746F5F6D61780A353A09776847
:1006300065656C5F6D61785F73706565640A363AF5
:1006400009776865656C5F74696D655F746F5F6D70
:1006500061780A0A703A097072696E742076616C6A
:100660007565730A643A097365742064656661751B
:100670006C74730A75703A092B310A646F776E3A9D
:10068000092D310A706775703A092B31300A70678D
:10069000646F776E3A092D31300A0A7370656564AC
:1006A000203D2064656C7461202A206D61785F7341
:1006B00070656564202A2028726570656174202F3A
:1006C0002074696D655F746F5F6D6178290A003F02
:1006D000004D3E2000433E20004C25640A00746912
:1006E0006D65725F72656164333228293A20253066
:1006F000346C580A006B6579626F6172645F69647B
:100700006C653A2025580A006B6579626F617264E6
:100710005F70726F746F636F6C3A2025580A0068BF
:100720006F73745F6B6579626F6172645F6C65642F
:100730007328293A2025580A000A092D205374618C
:10074000747573202D0A004743433A20342E392E06
:1007500032204156522D4C4942433A20312E382EF8
:100760003073766E204156525F415243483A2061C1
:100770007672350A004F5054494F4E533A204C552B
:100780004641204D4F5553454B45592045585452ED
:10079000414B455920434F4E534F4C4520434F4DFD
:1007A0004D414E4420343039360A004255494C44BC
:1007B0003A2022302E362E3332382D3437372D67FB
:1007C0003339383461312D646972747922202831CB
:1007D000353A30313A3538204A756E20203620328D
:1007E000303139290A005649443A20307846454587
:1007F00044284661746529205049443A20307830B5
:1008000030303028617269737529205645523A207C
:100810003078303030310A00444553433A20616C1F
:1008200069636520636F756E7465727061727420A0
:100830006B6579626F6172640A000A092D20566542
:100840007273696F6E202D0A000A092D20436F6EA6
:10085000736F6C65202D0A4553432F713A097175EA
:1008600069740A6D3A096D6F7573656B65790A0075
:100870000A092D204D61676963202D0A443A094415
:1008800065627567204D65737361676520546F6796
:10089000676C650A583A094D61747269782044653D
:1008A000627567204D6F646520546F67676C6520C3
:1008B0002D2053686F77206B65797072657373654F
:1008C0007320696E206D6174726978206772696443
:1008D0000A4B3A094B6579626F6172642044656224
:1008E000756720546F67676C65202D2053686F779C
:1008F000206B65797072657373207265706F7274A6
:100900000A4D3A094465627567204D6F757365201D
:10091000546F67676C650A563A0956657273696F5A
:100920006E0A533A095374617475730A433A094164
:100930006374697661746520436F6E736F6C6520B4
:100940004D6F64650A46312D4631303A0953776957
:1009500074636820746F204C6179657220302D3982
:100960002028463130203D204C30290A302D393A9C
:100970000953776974636820746F204C61796572DC
:1009800020302D390A47524156453A095377697448
:10099000636820746F204C61796572203020286173
:1009A0006C7465726E617465290A423A094A756D04
:1009B0007020746F20426F6F746C6F616465720A8F
:1009C0004553433A094A756D7020746F20426F6F2A
:1009D000746C6F616465722028616C7465726E61FD
:1009E0007465290A453A095072696E74204545506C
:1009F000524F4D2053657474696E67730A425350A9
:100A00004143453A09436C65617220454550524F58
:100A10004D0A000A002575002E6E6B726F3A200099
:100A20000A002575002E737761705F6261636B73D6
:100A30006C6173685F6261636B73706163653A20B8
:100A4000000A002575002E737761705F677261760A
:100A5000655F6573633A20000A002575002E6E6F8E
:100A60005F6775693A20000A002575002E7377616B
:100A7000705F72616C745F726775693A20000A007A
:100A80002575002E737761705F6C616C745F6C67A5
:100A900075693A20000A002575002E636170736C39
:100AA0006F636B5F746F5F636F6E74726F6C3A200D
:100AB000000A002575002E737761705F636F6E7496
:100AC000726F6C5F636170736C6F636B3A20000AC6
:100AD0000025303258006B65796D61705F636F6E11
:100AE0006669672E7261773A20000A002575002E2C
:100AF0006D6F7573653A20000A002575002E6B65D1
:100B000079626F6172643A20000A002575002E6DCB
:100B100061747269783A20000A002575002E656EAE
:100B200061626C653A20000A002530325800646525
:100B30006275675F636F6E6669672E7261773A20D0
:100B4000000A0025750064656661756C745F6C61F0
:100B50007965723A20003F000A6D6F7573653A201F
:100B60006F66660A000A6D6F7573653A206F6E0ACC
:100B7000000A6B6579626F6172643A206F66660A7B
:100B8000000A6B6579626F6172643A206F6E0A00C9
:100B90000A6D61747269783A206F66660A000A6DA0
:100BA00061747269783A206F6E0A000A6465627532
:100BB000673A206F66660A000A64656275673A20C4
:100BC0006F6E0A000A0A4A756D70696E6720746F4D
:100BD00020626F6F746C6F616465722E2E2E200020
:100BE000433E2000436C656172696E672045455045
:100BF000524F4D0A006565636F6E6669673A0A0079
:100C00005B735D004B6579626F6172642073746120
:100C100072742E0A005B575D005B535D005B525D92
:100C2000005B445D005B435D000403300000000C8A
:100C3000036100720069007300750000000A03463A
:100C40000061007400650000000403090409025BF0
:100C500000030100A0FA09040000010301010009DA
:100C600021110100012240000705810308000A0943
:100C70000401000103000000092111010001228587
:100C8000000705820320000A090402000203000095
:100C90000009211101000122220007058303200021
:100CA00001070503032000011201100100000008E4
:100CB000EDFE00000100010203010631FF0974A1ED
:100CC000010975150026FF00952075088102097637
:100CD000150026FF00952075089102C00501090244
:100CE000A10185020901A1000509190129051500C5
:100CF00025019505750181029501750381010501A5
:100D0000093009311581257F95027508810609385A
:100D10001581257F950175088106050C0A38021595
:100D200081257F950175088106C0C005010980A154
:100D30000185031601002603001A81002A8300752D
:100D40001095018100C0050C0901A101850416015F
:100D500000269C021A01002A9C0275109501810050
:100D6000C005010906A101050719E029E7150025BD
:100D70000195087501810295017508810105081921
:100D800001290595057501910295017503910105EC
:100D900007190029FF150026FF0095067508810038
:100DA000C00011241FBECFEFDAE0DEBFCDBF04B616
:100DB00003FE27C08091570290915802A0915902DA
:100DC000B0915A028730904BA740B04BD1F41092AB
:100DD0005702109258021092590210925A0214BEF1
:100DE00084B7877F84BF0FB6F894A8958091600080
:100DF000886180936000109260000FBEE0E0F8E32D
:100E0000099511E0A0E0B1E0EEE2FDE502C0059039
:100E10000D92A637B107D9F722E0A6E7B1E001C0ED
:100E20001D92A735B207E1F70E94A9280C94952ED0
:100E30000C940000FF93EF93E0917601F09177011D
:100E4000309709F00995EF91FF910895FC01859184
:100E5000803011F0EFDFFBCF0895FF27E0E230E2B2
:100E600047FF0CC0419597FF09C0EDE26095709572
:100E700080959095611D711D811D911D27FF02C0F8
:100E8000219530E350E2AA27660F771F881F991F2C
:100E9000AA1FA41710F0A41B63955A95A9F7AA30AE
:100EA00008F0A95FA05DAF93F39561157105810509
:100EB000910541F7ED3211F4EF93F395F21718F421
:100EC0003F93F395FBCF8F91B5DFFA95E1F7089546
:100ED000E991F9918591803021F0853219F0AADFEE
:100EE000F9CF089520E0E89455915532C1F350337D
:100EF00011F4689455915A3348F4505390F3220FEB
:100F0000022E220F220F200D250FF4CF0EF4219573
:100F100089919991533619F3533729F1533559F182
:100F2000BC0188279927E8945C3621F4899199912E
:100F300068945591543639F446EF7EF077FF0DC032
:100F40008FEF9FEF0AC055374AE039F0583540E13E
:100F500021F0523642E009F00895FF93EF937DDFD0
:100F6000EF91FF91B7CFFF93EF93FC018191803018
:100F7000B9F360DFFBCFFF93EF9368DFF1CFDF932F
:100F8000CF93CDB7DEB72596A3DFCF91DF9108953C
:100F90000C94320C0C94330C0C9461080C94A7083C
:100FA0000F931F93CF93DF939C013A9521153F41F7
:100FB00048F5EB018C0190FF03C080EEFB01099521
:100FC00011FF03C081EEFE01099512FF03C082EEFE
:100FD000FE01099513FF03C083EEFE01099501157B
:100FE000104180F084EEFE01099585EEFE01099521
:100FF00086EEFE01099587EEFE01DF91CF911F91EC
:101000000F910994DF91CF911F910F9108958770EF
:1010100091E001C0990F8A95EAF7892F0E94D41BAD
:101020000C940D1C877091E001C0990F8A95EAF726
:10103000892F0E94D41B0C940D1C877091E001C075
:10104000990F8A95EAF7892F0E94DA1B0C940D1CE0
:10105000877091E001C0990F8A95EAF7892F0E9465
:10106000DA1B0C940D1CCF93DF93EC01805E910989
:10107000089710F0209719F462E178E002C067E069
:1010800078E0CE010E94D0078C2FDF91CF910C9495
:101090009E11CF93DF93EC010E94D712CE01805EA8
:1010A0009109089710F0209719F468E278E002C0DF
:1010B0006DE178E0CE01DF91CF910C94D00781E013
:1010C000089581E008951F93CF93DF9300D000D05F
:1010D0001F92CDB7DEB749835A832091A60189813B
:1010E0009A81211112C0662349F00E943E1B182FDD
:1010F000682F89819A810E94E31A03C00E94121B03
:10110000182F69817A81812F04C00E943E1B69815A
:101110007A810F900F900F900F900F90DF91CF91E9
:101120001F910C94C109FC0140815181628173813E
:1011300084810C9463080E94A61C811102C00E9445
:10114000201D0C94C8070E94D70E0C94CA0708955E
:101150000C94CE0708950E9409160E94AA082FEF4A
:1011600084E39CE0215080409040E1F700C0000003
:101170000C944E1E0F931F93CF93DF938C010E940C
:101180009308EC01B8010E94370EB801CE010E940D
:10119000CC07882309F4EAC0B801CE010E947B0E77
:1011A000882309F4E3C0B801CE010E94910F88237F
:1011B00009F4DCC0C531FCE5DF0708F087C0C230A8
:1011C0008CE5D80708F452C0F8018281882309F41D
:1011D00054C00E94A61C811102C00E94201D0E94C2
:1011E000B91C90E09093490280934802FE01E350BD
:1011F000FC45E231F10530F4EA5AFF4F8091480294
:101200000C94392E80914802816027C0826025C0ED
:10121000846023C0806121C080621FC080641DC0C3
:1012200080681BC08460886018C08E7F16C08D7F68
:1012300014C08B7F12C08F7E10C08F7D0EC08F7B3D
:101240000CC08F770AC08B7F877F07C087FB222760
:1012500020F991E0922790FB87F9809348028091D2
:1012600048020E94BD1C0E94091680C0C115ECE511
:10127000DE0751F0C130DC4579F0C801DF91CF9134
:101280001F910F910C945F08F801C281CC2309F4DF
:101290006EC00E94AB086AC0F801C281CC2309F479
:1012A00066C080912602C82FC095C170C0FB80F92E
:1012B00080932602CC2329F08EE193E00E9426073A
:1012C00055C08CE093E00E94260751C0CC3D8CE5D0
:1012D000D80739F4F801C281CC2309F448C080E072
:1012E0000DC0CD3DECE5DE0760F0CD3D8CE5D807C7
:1012F00099F5F801C281CC23D1F182E00E945129F5
:1013000035C0C631DC4509F0B8CF0E94BE1B282F7E
:10131000F80182814091350150913601882379F09E
:101320002A7A91E009F490E090937801911102C03B
:1013300069E201C065E3CA010E94541D0AC08091A0
:101340007801811102C069E201C065E3CA010E940F
:10135000561D0E940D1C0AC0CE3DDC4509F08DCF04
:10136000F801C281CC2319F00E94201DC0E08C2F0F
:10137000DF91CF911F910F91089580E090E0089543
:1013800008959FE0799FF00111249BE4899FE00D6F
:10139000F11D1124E60FF11DEE0FFF1FE65BFE4F5E
:1013A000859194910895880F991FFC01E15DFC4F90
:1013B000859194910895CF93DF930E94C1090E9473
:1013C000920BEC01811520E59207F0F5811530E4D0
:1013D000930708F024C1883E910500F5803E9105F1
:1013E00008F09CC1883A910570F4853A910508F09F
:1013F0009FC08130910509F491C108F442C104975E
:1014000008F08CC13EC18F3B910508F49CC0803C24
:10141000910508F436C1805C9109F4C0811540E261
:10142000940758F4C11581E0D80708F077C1C03F90
:10143000D10508F426C1D06571C1811520E392075A
:1014400008F0E4C09F70DEC0811535E5930708F011
:1014500044C0811544E5940708F0F8C0C11582E541
:10146000D80708F5C11521E5D20708F0DBC08C2F9D
:10147000837021E030E002C0220F331F8A95E2F72B
:101480003C68CE0174E0969587957A95E1F7837074
:10149000382BCF70C695C69580E2C89FE001112415
:1014A000C22BD32B3BC12C2F26952695CE018370C2
:1014B0009927C115D34508F0BAC040E2249F900196
:1014C0001124C1E0D0E002C0CC0FDD1F8A95E2F705
:1014D0002C2B3D2BE901DC6821C1811549E59407DE
:1014E000A0F4C11588E5D80708F0B5C0C11526E5F8
:1014F000D20708F0C6C08C2F0E940F0C8F71C82F26
:10150000D0E0DC2FCC27D06209C181153AE59307E2
:1015100008F4A6C090568115904208F0B2C08D2FF5
:101520008F710E940F0CDD27D0628F71D82BF6C00F
:10153000853A910509F4A8C0863A910509F0A7C03B
:10154000C2E8D0E4EBC0883A910509F4A3C0893A17
:10155000910509F4A2C08A3A910509F4A1C08B3A19
:10156000910509F4A0C08C3A910509F49FC08B3B0A
:10157000910509F49EC08C3B910509F49DC08D3AFC
:10158000910509F49CC0803B910509F49BC08E3AFB
:10159000910509F49AC08F3A910509F499C0813BED
:1015A000910509F498C0823B910509F497C0833BEB
:1015B000910509F496C0843B910509F495C0853BDB
:1015C000910509F494C0863B910509F493C0873BCB
:1015D000910509F492C0883B910509F491C0893BBB
:1015E000910509F490C08D3B910509F48FC08E3BA5
:1015F000910509F48EC08A3B910509F48DC0C0E0C5
:10160000D4E48CC00E94D309EC0188C09927D3FF91
:1016100003C0EC01D86C82C0EC01D06C7FC0DF70DD
:10162000D06A7CC0DC2FCC27C16FD06A77C040E283
:10163000249F90011124C1E0D0E002C0CC0FDD1F37
:101640008A95E2F7C22BD32BDA6868C0D82FCC2753
:10165000C46FD06A63C0DC2FCC27C06FD06A5EC075
:101660008F700E940F0C94E0D695C7959A95E1F77C
:10167000CF70D0E0DC2FCC27D06A8F70806EC82B63
:101680004DC0C0E0D0E04AC0C1E8D0E447C0C3E8E4
:10169000D0E444C0C2EED4E441C0C9EED4E43EC0BC
:1016A000CAEED4E43BC0C5EBD4E438C0C6EBD4E406
:1016B00035C0C3EBD4E432C0C4EBD4E42FC0C7EBD5
:1016C000D4E42CC0CCECD4E429C0CDECD4E426C0C6
:1016D000C3E8D5E423C0CAE8D5E420C0C2E9D5E414
:1016E0001DC0C4E9D5E41AC0C1E2D6E417C0C3E204
:1016F000D6E414C0C4E2D6E411C0C5E2D6E40EC0FC
:10170000C6E2D6E40BC0C7E2D6E408C0CFE6D4E414
:1017100005C0C0E7D4E402C0CAE2D6E4CE01DF913E
:10172000CF9108958238910549F1B0F48133910544
:1017300009F458C048F48932910509F44EC08A3240
:10174000910509F454C008958533910509F440C00A
:101750008933910599F00895833E910529F138F474
:10176000803E910591F0823E9105A1F00895863E5C
:101770009105F9F0873E910531F1089520914802D5
:1017800020FD3AC021FD38C008958091480280FDB7
:1017900035C032C08091480282FF32C08091480239
:1017A00084FD30C083EE39C08091480282FD28C09C
:1017B000F5CF8091480283FF27C08091480284FDC5
:1017C00021C087EE2AC08091480283FD1DC0F5CF5D
:1017D0008091480285FD1AC01BC08091480285FD9A
:1017E00017C014C08091480286FD14C015C08091B6
:1017F000480286FD11C00EC080EE0FC089E30DC007
:1018000082EE0BC080E009C086EE07C089E205C009
:1018100085E303C08AE201C081E390E008959091DE
:10182000480292FF0DC0282F2871283019F4877FB5
:10183000846006C0282F2471243011F48B7F8860C7
:1018400093FF0DC0282F2871283119F4877E8461F9
:1018500006C0282F2471243111F48B7E886194FDF9
:10186000877E089508950895E82FF0E0EE0FFF1F9A
:10187000E758FE4F808191810895CF92DF92EF92D9
:10188000FF920F931F93CF93DF938FE393E00E9418
:10189000260789E7E82E81E0F82EC0E0D0E09AE341
:1018A000C92E93E0D92E01E313E0DF93CF93DF92AB
:1018B000CF920E94BF0787E393E00E942607F701BB
:1018C000819191917F010E948C1C9F938F931F9314
:1018D0000F930E94BF078FE293E00E942607219694
:1018E0008DB79EB708960FB6F8949EBF0FBE8DBFFA
:1018F000C530D105D1F6DF91CF911F910F91FF90A7
:10190000EF90DF90CF900895E7E5F1E041E050E0FF
:1019100025E02E0F9191A92FA295AF70B0E091967E
:101920003C9191979F70BA0102C0660F771F9A95FC
:10193000E2F7CB018095832391968C932E13EACF07
:10194000A8E4B1E041E050E02FE02A0F8D91E82FAC
:10195000E295EF70F0E031A18F70BA0102C0660F1E
:10196000771F8A95E2F7CB01962F9095932391A349
:1019700092A1892B82A32A13E9CFE3E8F1E0A9E73A
:10198000B1E0119211921D921D9271E0ED38F707AE
:10199000C1F785E00E94650D0C949B085F926F92E1
:1019A0007F928F929F92AF92BF92CF92DF92EF92EF
:1019B000FF920F931F93CF93DF9307E511E0A3E806
:1019C000B1E0612CEE24E394F12C5D018D909C90AC
:1019D000119711961C921E92E80189918E01E82FB1
:1019E000E295EF70F0E091A18F70A70101C0440F64
:1019F0008A95EAF7892F842B81A382A1542E5094D3
:101A0000852182A3D0EADA95F1F788E4C82E81E037
:101A1000D82E80E090E0E60179906E01272D229586
:101A20002F7030E0E90168A12D913C91119770E091
:101A3000D72DDF7002C075956795DA95E2F760FDE6
:101A400008C0B701082E02C0660F771F0A94E2F79C
:101A500002C060E070E0262B372B11963C932E934A
:101A600001968F309105B9F681A1D52DD823D1A348
:101A700082A1482B42A3129681E0F5012081318199
:101A80008216930609F480E0682AF1E0AD38BF07BA
:101A900009F09BCF262D45E069E771E083E891E0EE
:101AA0000E94660D0E94A308862DDF91CF911F91A1
:101AB0000F91FF90EF90DF90CF90BF90AF909F90ED
:101AC0008F907F906F905F9008950895FF920F938D
:101AD0001F93CF93DF93F82E092F162FD72FC42FE4
:101AE000222349F081E080938F010E94E61D9093AC
:101AF0008E0180938D0180918F018823D9F0809190
:101B00008D0190918E010E94FE1D069798F0EF2D99
:101B1000F02FA12FBD2F80E090E04C2F50E08417D4
:101B2000950734F4219131912D933D930196F7CF90
:101B300010928F01DF91CF911F910F91FF90089527
:101B4000CF93DF93FC012189211116C0EC0181E0C4
:101B5000818B87810E94C11B88850E94D41B0E94B3
:101B60000D1CEA81FB816C897D89CE010696309738
:101B700019F0DF91CF910994DF91CF910895CF9320
:101B8000DF93FC012081223041F4FB01EC018281D2
:101B900093810E94330881E08B87DF91CF91089574
:101BA000FC018081813021F4FB018081918105C09D
:101BB000823029F4FB01828193810C9433080895CB
:101BC000FC018081813021F4FB018081918105C07D
:101BD000823029F4FB01828193810C944908089595
:101BE000EF92FF920F931F93CF93DF93FC01228517
:101BF000211136C0EC01E380F480F7E5FF1A26E1FD
:101C00002E9DC0012F9D900D1124DC01A050BF4FCF
:101C10001496ED91FC91159754966D917C91559782
:101C20008A5F9E4F309709F0099586E18E9D80016D
:101C30008F9D100D112400501F4FF80187810E94C5
:101C4000C71BF80180850E94DA1B0E940D1C1882B8
:101C500019861B861E821D8210929101109290019E
:101C6000DF91CF911F910F91FF90EF900895DF9238
:101C7000EF92FF920F931F93CF93DF93FB0122818B
:101C8000222389F1209134012F3F69F18C01C6E0B4
:101C9000D1E0E12CF12CDD24D39480913401082E85
:101CA000000C990B8E159F05F4F088818823B1F004
:101CB0008B819C810817190739F4809190019091CC
:101CC00091010817190751F0D9861E830D83CE01A3
:101CD00006970E94A00DCE010E94F00DFFEFEF1AB3
:101CE000FF0A6696DACFDF91CF911F910F91FF9097
:101CF000EF90DF900895EF92FF920F931F93CF9391
:101D0000DF939C0137552F3F310511F008F047C094
:101D100040913401042E000C550B4217530714F464
:101D200020933401FB017C01828196E1929F800126
:101D3000939F100D1124E801C050DF4F888B9281D2
:101D40008E81992311F1FA86E9868F5F8E830E9436
:101D5000E61D9E878D870E94F41B8F830E94BE1B09
:101D600088870E94D11B9885892B8887E881F98113
:101D70006C897D89C8018A5F9E4F309709F009956B
:101D8000F0929101E09290010AC0882341F0898984
:101D9000882329F0C8018A5F9E4F0E94F00D81E0E0
:101DA000DF91CF911F910F91FF90EF900895CF9207
:101DB000DF92EF92FF920F931F93CF93DF93809167
:101DC00034018F3FC1F1C0E0D6E12C2F30E080918B
:101DD0003401082E000C990B8217930764F1D29FEF
:101DE000F001D39FF00D1124E050FF4FE288F388FB
:101DF000E114F10419F488ECE82EF12CD29F600173
:101E0000D39FD00C1124860100501F4FF80186810A
:101E1000882379F0858596850E94FE1DE816F906CF
:101E200040F4C8010E94A00DC6018A5F9E4F0E9427
:101E3000F00DCF5FCACFDF91CF911F910F91FF902F
:101E4000EF90DF90CF9008950F931F93CF93DF9380
:101E5000C62FD42F022FFC0182818823C9F0609302
:101E600094010E94E61D909393018093920180E279
:101E70008C0F883008F050C0C77081E001C0880F17
:101E8000CA95EAF7DF91CF911F910F910C945213ED
:101E900010919401161330C080919201909193019A
:101EA0000E94FE1D883C910538F5C0E2CD0F1D173C
:101EB000B9F080E2810F883040F4177081E001C0F2
:101EC000880F1A95EAF70E945913C83048F481E048
:101ED0009D2F977001C0880F9A95EAF70E945213C0
:101EE000802F0E943F13C830B8F4D77081E001C042
:101EF000880FDA95EAF70AC080E28C0F883060F428
:101F0000C77081E001C0880FCA95EAF7DF91CF91D1
:101F10001F910F910C945913DF91CF911F910F9145
:101F200008959C01CB01203F4CE53407F9F078F48B
:101F3000283DFCE53F07B9F0293D4CE5340711F198
:101F4000273D3C4531F526E241EE61EE1EC0223FC1
:101F5000FCE53F0799F070F0233F3C45D1F427E2C0
:101F600045EE66EE12C027E245EE0EC026E241EED7
:101F700060EE0BC027E245EE64EE07C026E241EEBC
:101F800062EE03C028E241E065EE0E94240F80E08B
:101F90000895FC018281882319F01092940108951C
:101FA00081E0089590939A01809399010895E091BA
:101FB0009901F0919A01309721F00190F081E02D84
:101FC000099480E00895EF92FF920F931F93CF93AF
:101FD000DF93E0919901F0919A013097B1F18C0172
:101FE0000280F381E02D09958091260282FF2DC0A9
:101FF00080FF04C08EE593E00E942607E80118E008
:1020000088E5E82E83E0F82E8091260280FF0BC041
:1020100088811F928F93FF92EF920E94BF070F90CB
:102020000F900F900F90115021961111EDCF8091CC
:10203000260280FF0AC086E593E0DF91CF911F91D1
:102040000F91FF90EF900C942607DF91CF911F9195
:102050000F91FF90EF900895E0919901F0919A010E
:10206000309739F022E0DC012C930480F581E02DDB
:102070000994089520919701309198018217930750
:1020800071F09093980180939701E0919901F091FC
:102090009A01309721F00680F781E02D0994089588
:1020A00020919501309196018217930771F09093DA
:1020B000960180939501E0919901F0919A013097F2
:1020C00021F00084F185E02D0994089585B780689A
:1020D00085BF85B7806885BF0895089508950C94DD
:1020E0006E1008950C9471100E9466100E946D107D
:1020F0000C946F1081E008950E94DD1D0E94840CF5
:102100000E94721E0C947210CF93C82F80912602E9
:1021100082FF1EC080FF04C087E793E00E9426076D
:102120008091260280FF0CC01F92CF9382E793E03C
:102130009F938F930E94BF070F900F900F900F9067
:102140008091260280FF04C080E793E00E9426076A
:102150008C2FCF910C94A8084F925F927F928F9210
:102160009F92AF92BF92CF92DF92EF92FF920F9326
:102170001F93CF93DF93CDB7DEB72A970FB6F894AE
:10218000DEBF0FBECDBF0E94CE0C0E947A1081111F
:1021900011C08FEF89838A831B820E94E61D8160B4
:1021A000782F9D838C8349815A816B818D810E9418
:1021B0006A1157C09CE9C92E91E0D92E00E010E0C9
:1021C000AA24A394B12C702E802F0E94340C4C01B1
:1021D000F601419051906F0148265926411451044F
:1021E00031F40F5F1F4F0530110569F7D2CF809191
:1021F000260281FD0E943D0C20E030E07501022E98
:1022000002C0EE0CFF1C0A94E2F7C701842195215D
:10221000892B09F12E837F828E209F2091E08928CF
:1022200009F490E098870E94E61D8160782F9A87D4
:1022300089874E815F8168858A850E946A11000FB7
:10224000111FF801E456FE4F80819181E826F9269E
:10225000F182E08206C02F5F3F4F2F30310571F6CB
:10226000C0CF0E94872010919B010E94D70F1817A2
:10227000D9F00E94D70F80939B012A960FB6F8944D
:10228000DEBF0FBECDBFDF91CF911F910F91FF90A9
:10229000EF90DF90CF90BF90AF909F908F907F9006
:1022A0005F904F900C9484102A960FB6F894DEBF7E
:1022B0000FBECDBFDF91CF911F910F91FF90EF9097
:1022C000DF90CF90BF90AF909F908F907F905F9066
:1022D0004F900895CF93DF93CDB7DEB72B970FB60E
:1022E000F894DEBF0FBECDBF4F83588769877A87CA
:1022F0008B87DE01119686E0FD0111928A95E9F740
:1023000085E0FE01379601900D928A95E1F74981AB
:102310005A816B817C818D819E810E94B3182B969E
:102320000FB6F894DEBF0FBECDBFDF91CF910895F9
:10233000FC01808191810E947F1B0895CF93DF93E0
:102340001F92CDB7DEB7882309F42DC1682F8238DC
:10235000C1F40E94D70F81FD26C169E38091350148
:10236000909136010E94541D0E940D1C2FEF81EEAA
:1023700094E0215080409040E1F700C0000069E304
:1023800019C0833811F50E94D70F80FD0CC163E599
:1023900080913501909136010E94541D0E940D1CC0
:1023A0002FEF81EE94E0215080409040E1F700C093
:1023B000000063E580913501909136010E94561D21
:1023C0000F90DF91CF910C940D1C8438C1F40E94C2
:1023D000D70F82FDE8C067E4809135019091360106
:1023E0000E94541D0E940D1C2FEF81EE94E021509D
:1023F00080409040E1F700C0000067E4DBCF8CEF45
:10240000860F813A70F4862F69830E94F4246981D3
:102410008111C9C080913501909136010E94541DEF
:10242000CFCF80E2860F883048F4677081E001C02A
:10243000880F6A95EAF70E94C11BC2CF8BE5860F11
:10244000833088F4653A29F0663A31F083E890E009
:1024500005C081E890E002C082E890E00F90DF9133
:10246000CF910C943A1088E5860F873108F091C01F
:10247000683A09F445C0693A09F445C06A3A09F472
:1024800045C06B3A09F445C06C3A09F445C06B3B52
:1024900009F445C06C3B09F445C06D3A09F445C0E8
:1024A000603B09F445C06E3A09F445C06F3A09F43F
:1024B00045C0613B09F445C0623B09F445C0633B3C
:1024C00009F445C0643B09F445C0653B09F445C0C7
:1024D000663B09F445C0673B09F445C0683B09F415
:1024E00045C0693B09F445C06D3B09F445C06E3BEE
:1024F00009F445C06A3B09F445C080E090E044C05F
:1025000082EE90E041C089EE90E03EC08AEE90E01D
:102510003BC085EB90E038C086EB90E035C083EBA4
:1025200090E032C084EB90E02FC087EB90E02CC0AD
:102530008CEC90E029C08DEC90E026C083E891E01F
:1025400023C08AE891E020C082E991E01DC084E9BF
:1025500091E01AC081E292E017C083E292E014C0D9
:1025600084E292E011C085E292E00EC086E292E041
:102570000BC087E292E008C08FE690E005C080E7DC
:1025800090E002C08AE292E00F90DF91CF910C942C
:102590005010603F40F0862F0E940D1F0F90DF917A
:1025A000CF910C94FA1F0F90DF91CF91089588235B
:1025B00009F464C0823879F40E94D70F81FF5EC0AD
:1025C00069E380913501909136010E94541D0E946B
:1025D0000D1C69E310C08338B1F40E94D70F80FF4F
:1025E0004DC063E580913501909136010E94541DE4
:1025F0000E940D1C63E580913501909136010E9487
:10260000561D0C940D1C843879F40E94D70F82FF5C
:1026100035C067E480913501909136010E94541DC8
:102620000E940D1C67E4E7CF9CEF980F913A10F4DD
:10263000682FE1CF90E2980F983050F4877091E0C6
:1026400001C0990F8A95EAF7892F0E94C71BD9CF3D
:102650009BE5980F933020F480E090E00C943A10C2
:1026600098E5980F973120F480E090E00C9450109A
:10267000803F20F00E94751F0C94FA1F0895CF939D
:10268000C82F0E949E11C93349F42FEF83EC99E0C3
:10269000215080409040E1F700C000008C2FCF9186
:1026A0000C94D712882321F00E94C11B0C940D1C9E
:1026B0000895882321F00E94C71B0C940D1C0895D7
:1026C0004F925F926F927F92BF92CF92DF92EF9282
:1026D000FF920F931F93CF93DF937C01062FC72F99
:1026E000FC01158112951F70D281D1110E94E11B4E
:1026F0000E94B71B882379F0DD2369F080E2800F08
:10270000883048F082E00E94581C0E94B71B91E07C
:10271000B82EB92601C0B12CCC2EC2948FE0C822AD
:10272000D12CF601E859FF4F0C94392E8C2F807F65
:10273000CF70882311F0C295C07FDD2399F0CC23A0
:1027400009F4C3C180E2800F883010F0011104C089
:102750008C2F0E94C11B03C08C2F0E94D41B0E948F
:102760000D1CB3C1802F0E94D712CC2309F4D2C113
:1027700080E2800F883010F0011104C08C2F0E947D
:10278000C71B03C08C2F0E94DA1B0E940D1CC2C104
:102790008C2F807FCF70803211F0C295C07F0023D4
:1027A00019F00130C9F022C0DD2371F0112341F08E
:1027B000113031F40E94F41B8C2B0E94FA1BAAC129
:1027C0000E94F41B8C2B3AC1112319F0113009F42B
:1027D000A1C10E94031C18C0DD2321F0163008F0AF
:1027E00099C10EC0153008F095C10EC0DD2351F01F
:1027F000112331F0F701858180FF67C18F708583D8
:102800008C2F1CC1111172C18C2F1EC18C2F86956B
:102810008695837090E0009719F0019761F07AC176
:10282000DD2321F0802F9C2F937002C080E090E088
:102830000E943A107FC1DD2321F0802F9C2F9370DE
:1028400002C080E090E00E94501074C1DD23F9F0D6
:10285000053F51F0063F71F0043FA9F48091420218
:102860009091430281600BC080914202909143029B
:10287000826005C0809142029091430284609093EF
:10288000430280934202802F0E940D1F1EC0053F0D
:1028900051F0063F71F0043FA9F4809142029091FB
:1028A00043028E7F0BC080914202909143028D7F44
:1028B00005C080914202909143028B7F9093430226
:1028C00080934202802F0E94751F0E94FA1F32C11E
:1028D0008C2F837009F04BC0D11128C1202F229575
:1028E00026952770220F220F602F6F70862F90E0A1
:1028F000A0E0B0E02C013D01022E04C0440C551CA8
:10290000661C771C0A94D2F704FF10C08FE090E099
:10291000A0E0B0E004C0880F991FAA1FBB1F2A9532
:10292000D2F780959095A095B09503C080E090E097
:10293000DC01C695C695C370D0E0BC01CD01642909
:10294000752986299729C230D10559F0C330D105A0
:1029500059F0219719F00E94F819E8C00E94E61971
:10296000E5C00E940A1AE2C00E94E419DFC0DD231C
:1029700019F08C2F817001C08695882309F4D6C088
:10298000202F229526952770220F220F602F6F701F
:10299000862F90E0A0E0B0E02C013D01022E04C0A3
:1029A000440C551C661C771C0A94D2F704FF10C017
:1029B0008FE090E0A0E0B0E004C0880F991FAA1F4C
:1029C000BB1F2A95D2F780959095A095B09503C02E
:1029D00080E090E0DC01C695C695C370D0E0BC01F4
:1029E000CD016429752986299729C230D10559F06E
:1029F000C330D10559F0219719F00E94BE1A96C034
:102A00000E94AC1A93C00E94D01A90C00E941F1A54
:102A10008DC0802F90E0FC01E05EF109E531F10509
:102A200008F04FC0E858FF4F0C94392E0F708C2FD0
:102A30008F71DD2331F00E94451A802F0E945213BE
:102A400069C00E94661A802F0E94591363C0DD235B
:102A500041F0153008F05EC08C2F8F710E948B1AE8
:102A600059C0163008F056C0F7CFDD2339F08C2F4F
:102A70008F710E94451A4EC0DD23C9F38C2F8F71D0
:102A80000E94661A47C0DD2329F08C2F8F710E94A7
:102A9000301A40C00E942B1A3DC0DD2349F0CF718F
:102AA0008C2F0E94451A63E08C2F0E94431C32C079
:102AB00081E00E94581C123068F182E00E94581C8C
:102AC00029C0DD2331F0112391F2802F0E949E1145
:102AD00021C0112399F2093349F4FFEF23EC89E077
:102AE000F15020408040E1F700C00000802F0E949C
:102AF000D71210C04C2F4F70602FC7010E94BD0924
:102B00000E94571917C04C2F4F70602FC7010E94A9
:102B1000C00910C098E0C916D10441F05CF0FAE099
:102B2000CF1AD10822E0C216D10420F40E94D70F98
:102B30000E94A808BB20F1F00E94B31B80FD1AC0C0
:102B4000F70112820E94AD1B0E94451AC7010E9424
:102B5000C8150E94AD1BDF91CF911F910F91FF907F
:102B6000EF90DF90CF90BF907F906F905F904F90ED
:102B70000C94661ADF91CF911F910F91FF90EF9007
:102B8000DF90CF90BF907F906F905F904F900895AF
:102B90000F931F93CF93DF93EC01888199812B8151
:102BA0003C81232BB9F09F3F11F48F3F99F0CE0168
:102BB0000E94BA08882371F0688179818A810E9415
:102BC0008A1B8C010E94E21A0E94E319B801CE010F
:102BD0000E946013DF91CF911F910F9108950E9481
:102BE000E11B0E94F11B0E940D1C0E9422210E94E9
:102BF000FA1F80E090E00E943A1080E090E00C9490
:102C0000501080913501909136010E94581D0C940E
:102C1000EF150E94CE1B0C940116E92FE295EF7080
:102C2000F0E03297EE30F105B0F4E357FF4F0C942B
:102C3000392E803F91F018F4803E68F40EC0843F36
:102C400051F40BC0803E48F0813F29F406C093FB4D
:102C5000882780F9089580E0089581E008950E9412
:102C60007F1B0E940D160895CF93DF9300D000D0F4
:102C70001F92CDB7DEB70F900F900F900F900F906F
:102C8000DF91CF910895CF93DF9300D000D000D093
:102C9000CDB7DEB726960FB6F894DEBF0FBECDBF18
:102CA000DF91CF9108951F93CF93DF93C091A70138
:102CB00016E08091A801C81799F0D0E01C9FF001A0
:102CC0001D9FF00D1124E755FE4F40815181628117
:102CD0007381848195810E9443162196C770E9CF44
:102CE000DF91CF911F9108954091D9015091DA0160
:102CF0006091DB017091DC018091DD019091DE013A
:102D00000C9443168091DE0182958F7009F054C0B7
:102D10008091DB01882309F44FC08091A701A09125
:102D2000A8016091D9017091DA014091DC015091C4
:102D3000DD01B6E08A1709F43FC090E04115510566
:102D4000C1F17F3F11F46F3FA1F1B89FF001B99F2E
:102D5000F00D1124E755FE4F218172132AC0208106
:102D6000621327C02281211124C0238134812417BA
:102D7000350710F421503109241B350B283C31054F
:102D8000C0F42091DE012F7020612093DE0126E047
:102D9000289FF001299FF00D1124E255FE4F8081FC
:102DA0008F708061808389ED91E00E94C8150C943A
:102DB000531601968770BECF0895CF92DF92EF929F
:102DC000FF920F931F93CF93DF93CDB7DEB7629738
:102DD0000FB6F894DEBF0FBECDBF8C0185E0F801C1
:102DE000DE011D9601900D928A95E1F7D8014C9174
:102DF00011965C91119712966C9112971396CD9043
:102E0000DC9014973091D9017091DA018091DC0146
:102E10009091DD01009709F46BC17F3F19F43F3FAA
:102E200009F466C1E090DB01EE2009F4C0C02091F6
:102E3000DE01C816D90628F0F601E81BF90BCF0110
:102E400004C0809590958C0D9D1DFF24F394883CC3
:102E5000910578F0F12C207F09F0C6C07C2DD98A2D
:102E6000C88A89890E94341689ED91E00E94C815AC
:102E7000B1C0822F807F09F046C0751314C034138F
:102E800012C0611110C02F7020612093DE010E94DA
:102E9000741689ED91E00E94C8158091DE01D80179
:102EA00015968C932EC0CD2819F15F3F11F44F3F3A
:102EB000F9F0F62E61111CC08091A7012091A801A4
:102EC00036E0821709F45AC090E0389FF001399F2C
:102ED000F00D1124E755FE4F7181571306C0708124
:102EE000471303C07281711103C001968770E9CF47
:102EF000F62E662309F427C18091DE01816080935C
:102F0000DE01F12C20C1751308C0341306C0611115
:102F100004C08091DE01D801C3C04D875E878D85D6
:102F20009E856A8B0E942F166A898823E1F16623A9
:102F3000D1F12091DE01822F82958F7090E002976F
:102F400074F08091D9019091DA0198878F83198666
:102F5000DB86CA862C87CE0107960E94C81586E0BC
:102F6000F801A9EDB1E001900D928A95E1F70E9478
:102F700082160E947416FF24F394E5C04D875E8785
:102F80008D859E850E947F1B292F22952F7030E012
:102F9000223031050CF0CBC09F7009F0C5C0805EB7
:102FA000883008F4D0C0C8010E94C815E4CFC81604
:102FB000D90608F453C0F601E81BF90BCF01883C91
:102FC000910508F450C0F12C7C2DD98AC88A8989D2
:102FD0000E943416E9EDF1E086E0DF011D928A954A
:102FE000E9F70E947416AFC0751314C0341312C0F1
:102FF000611110C08091DE01F8018583C8010E9433
:10300000C81586E0E9EDF1E0DF011D928A95E9F748
:10301000FE2C99C04D875E878D859E856A8B0E94A8
:103020002F166A89882309F4BECF662309F4BBCF23
:103030002091DE01822F82958F7090E002970CF430
:103040008ECF8091D9019091DA019A8389831B8276
:10305000DD82CC822E83CE0101967FCF8095909524
:103060008C0D9D1DACCFF62E662309F49CCF7513F5
:103070002EC034132CC02091DE0120FD1FC0822FF2
:1030800082958F70D9F0D80115962C9315978F30B3
:1030900049F08F5F982F9295907F822F8F70892BA8
:1030A00015968C93C8010E94C81586E0F801A9ED19
:1030B000B1E001900D928A95E1F793CF86E0F80197
:1030C000A9EDB1E001900D928A95E1F73CC04D87E2
:1030D0005E878D859E850E942F16811140CF80913D
:1030E000DE0181608093DE01C8010E94C8152BC0FB
:1030F000662309F458CF4D875E878D859E850E9493
:103100002F16F82E882309F44ECF86E0F801A9ED9A
:10311000B1E001900D928A95E1F789ED91E00E946E
:1031200098110E9482165DCF811139CF0CC02430D6
:1031300031050CF038CF9F7009F431CFF80195813B
:10314000907F09F02CCF8F2D62960FB6F894DEBFDA
:103150000FBECDBFDF91CF911F910F91FF90EF90E8
:10316000DF90CF9008951F93CF93DF93CDB7DEB755
:103170002C970FB6F894DEBF0FBECDBF4F83588794
:1031800069877A878B879C87CE0107960E94DD1618
:10319000882369F08F8198852A853B85232BF1F15F
:1031A0009F3F09F063C08F3F09F060C037C086E0E1
:1031B000FE013796DE01119601900D928A95E1F796
:1031C0006F817885EA85FB85309741F17F3F11F467
:1031D0006F3F21F12091A80130E0C901019687706D
:1031E00099274091A70150E08417950709F447C03B
:1031F00069837A83FD83EC8396E0929FD001939F4D
:10320000B00D1124A755BE4FFE01319601900D92CD
:103210009A95E1F78093A8010E94531616E08091D9
:10322000A7019091A8018917C1F1189FC00111242D
:1032300087559E4F0E94DD16882379F1E091A70102
:103240001E9FF0011124E755FE4F4081518162819C
:103250007381848195810E9443168091A70190E03B
:103260000196877099278093A701D9CF4F81588500
:1032700069857A858B859C850E944316CFCF0E94F5
:1032800009161092A8011092A701E9EDF1E086E07D
:10329000DF011D928A95E9F7C1CF2C960FB6F894FD
:1032A000DEBF0FBECDBFDF91CF911F910895EF928A
:1032B000FF920F931F93CF93DF938C01892B09F417
:1032C0006CC0F12CEE24E394E8012196F80184917E
:1032D000843740F4843008F051C0813081F082306E
:1032E00019F15BC0853709F444C0A8F19CE7980F39
:1032F000903708F052C08F770E94D71241C00E5FFE
:103300001F4FFE01C49180E28C0F883048F4C770D3
:103310008E2D01C0880FCA95EAF70E94E41B14C0E5
:103320008C2F0E949E112DC00E5F1F4FFE01C49175
:1033300080E28C0F883058F4C7708E2D01C0880F42
:10334000CA95EAF70E94EA1B0E940D1C1AC08C2F36
:103350000E94D71216C00E5F1F4FFE01C491CC23EE
:1033600081F08FE99FE00197F1F700C00000C150A4
:10337000F6CF0E5F1F4FFE01F49003C00E949E1116
:103380008E018F2D882309F49FCFEFE9FFE031975D
:10339000F1F700C000008150F5CFDF91CF911F9170
:1033A0000F91FF90EF90089508950C94D4190E9406
:1033B000D5196093150270931602809317029093AB
:1033C00018020C94EF1508950C94D7190F931F93BE
:1033D00000911502109116022091170230911802E7
:1033E000602B712B822B932B1F910F910C94D7196B
:1033F0000F931F930091150210911602209117024E
:103400003091180260237123822393231F910F911F
:103410000C94D7190F931F93009115021091160267
:103420002091170230911802602771278227932775
:103430001F910F910C94D71908950C941C1A0E9497
:103440001D1A6093110270931202809313029093DD
:1034500014020C94EF1560E070E0CB010C941F1A7D
:103460000F931F9341E050E060E070E08A019B0100
:1034700004C0000F111F221F331F8A95D2F7C90104
:10348000B8011F910F910C941F1A0F931F9341E0E5
:1034900050E060E070E004C0440F551F661F771FC6
:1034A0008A95D2F78091110290911202A091130295
:1034B000B09114028A019B01082B192B2A2B3B2B5C
:1034C000C901B8011F910F910C941F1A0F931F93FC
:1034D00041E050E060E070E004C0440F551F661FFB
:1034E000771F8A95D2F74095509560957095809199
:1034F000110290911202A0911302B09114028A015C
:103500009B01082319232A233B23C901B8011F91DA
:103510000F910C941F1A0F931F9341E050E060E04D
:1035200070E004C0440F551F661F771F8A95D2F7BD
:103530008091110290911202A0911302B091140295
:103540008A019B01082719272A273B27C901B801AF
:103550001F910F910C941F1A0F931F93009111024A
:10356000109112022091130230911402602B712BE2
:10357000822B932B1F910F910C941F1A0F931F9363
:103580000091110210911202209113023091140245
:1035900060237123822393231F910F910C941F1A90
:1035A0000F931F93009111021091120220911302A8
:1035B0003091140260277127822793271F910F9162
:1035C0000C941F1A08952FE0929F800D1124A82FAC
:1035D000A695A695A695877051E001C0550F8A95CE
:1035E000EAF785E0A89FD001112420E030E070E0E8
:1035F000F901EA0FFB1FE152FE4F4081CB01022E81
:1036000002C0969587950A94E2F781709927819573
:1036100084278523842780832F5F3F4F2530310502
:1036200039F708952FE0929F800D1124682F669539
:1036300066956695982F977085E0689FB001112474
:1036400040E050E080E0FA01E60FF71FE152FE4F44
:10365000208130E0092E02C0369527950A94E2F7C2
:1036600021703327042E01C0220F0A94EAF7822B1F
:103670004F5F5F4F4530510531F70895BF92CF92AC
:10368000DF92EF92FF920F931F93CF93DF938C0102
:10369000C0901502D0901602E0901702F090180228
:1036A0008091110290911202A0911302B091140224
:1036B000C82AD92AEA2AFB2ACFE1D0E0D701C601DD
:1036C0000C2E04C0B695A795979587950A94D2F7C6
:1036D00080FF07C0BC2EB8018C2F0E94DB09019728
:1036E00019F4219758F7B12C8B2DDF91CF911F91B1
:1036F0000F91FF90EF90DF90CF90BF900895CF9300
:10370000DF93EC010E943E1BBE010E94DB09DF91AA
:10371000CF9108951F93CF93DF93EB019091A60172
:10372000992321F0CB010E947F1B13C0882349F00D
:10373000CB010E943E1B182F682FCE010E94E31A76
:1037400004C0CB010E94121B182FBE01812F0E94C2
:10375000DB09DF91CF911F91089580911902859522
:1037600085958595089580911902877008959091A7
:103770001902977081E009F480E008958091250294
:10378000089590912502892B8093250208958095B4
:103790009091250289238093250208951092250295
:1037A000089580912402089590912402892B80939A
:1037B0002402089580959091240289238093240205
:1037C000089510922402089590912302892B8093EA
:1037D00023020895809590912302892380932302E8
:1037E000089510922302089580911A020895089571
:1037F0000C94F71B90911A02981721F080931A02EB
:103800000C94F81B089580911A02882329F01092D5
:103810001A0280E00C94F81B0895E0913501F091B4
:103820003601809125028083E0913501F0913601C7
:10383000908180912402892B8083E0913501F09161
:103840003601908180912302892B808380911A0216
:10385000882381F0E0913501F09136019081892B28
:10386000808380913501909136010E94221D811143
:103870000E94031C80913501909136010C94E30F56
:1038800008950C94401C98E0899F90011124262BE8
:10389000209319020E94451A8091190285958595F9
:1038A00085950C94411C1092190280E00C94411CE7
:1038B000209119028095822380931902982F977086
:1038C00079F430E0482F082E000C550B24173507EB
:1038D00039F08595859585950E94661A0C94531C40
:1038E0000895909377018093760108958295982F9B
:1038F0009C7C392F36953695282F237344E0249FDE
:10390000C0011124932F982B292F2A7A2695892FCD
:103910008575880F822B08951F93CF93DF931F9295
:10392000CDB7DEB799830E94761C182F9981892F15
:103930000E94761C212F30E0322F2227A901482B2C
:10394000CA010F90DF91CF911F91089580E090E020
:103950000E945B2E21E08D3E9E4F09F020E0822FD9
:10396000089582E090E00C94532E83E090E00C9454
:10397000532E84E090E00C94532E682F84E090E066
:103980000C94612EAB01BC018FE090E00C94732E7F
:10399000AB01BC0183E190E00C94732E60E070E019
:1039A000CB010C94C81C60E070E0CB010E94C21CEB
:1039B0000C94CE1C6DEE7EEF80E090E00E947F2E96
:1039C00060E082E090E00E94612E60E083E090E0A1
:1039D0000E94612E10921502109216021092170288
:1039E0001092180260E084E090E00E94612E60E096
:1039F00085E090E00E94612E60E086E090E00E9409
:103A0000612E6FEF87E090E00E94612E40E050E071
:103A1000BA0188E090E00E94732E60E08DE090E0B3
:103A20000E94612E40E050E0BA0188E190E00E94DF
:103A3000732E60E087E190E00E94612E0C94D31C0D
:103A40000C94DA1CFC01329697E080E0915029F04A
:103A500021912223D9F38F5FF9CF08959C01FC01B6
:103A600032969FEF80E04191461789F09F3F19F40D
:103A7000411101C0982F8F5F8630A9F79F3F39F021
:103A8000F901E90FF11D97FDFA95628308950895F4
:103A9000FC01329608962081261301C010823196CF
:103AA000E817F907C1F708950C942E1D0C94481DD2
:103AB000029626E0FC0111922A95E9F708950895EF
:103AC0000C945F1D0E94601D80914E02843049F16C
:103AD0001092270220E488E190E00FB6F894A895B0
:103AE000809360000FBE2093600080E00E94A808D1
:103AF0000E94601D83B7817F846083BF83B781602C
:103B000083BF7894889583B78E7F83BF0FB6F89470
:103B1000A895809160008861809360001092600099
:103B20000FBE089508950895CF930E94921D0E949C
:103B3000CE0C0E94931DC0E08C2F0E94340C892B68
:103B400029F4CF5FC530C1F780E001C081E0CF919B
:103B5000089508950C94A91D0E9409160E94D70F7C
:103B60000E94A8080C94AA1D1F920F920FB60F92E4
:103B700011248F939F93AF93BF938091270281115C
:103B800013C08091440290914502A0914602B091E9
:103B900047024196A11DB11D8093440290934502B6
:103BA000A0934602B0934702BF91AF919F918F912E
:103BB0000F900FBE0F901F90189582E084BD93E088
:103BC00095BD9AEF97BD80936E0008952FB7F89436
:103BD0008091440290914502A0914602B091470223
:103BE0002FBF08952FB7F894609144027091450259
:103BF00080914602909147022FBF0895CF92DF92A5
:103C0000EF92FF920F931F932FB7F89440914402C5
:103C10005091450260914602709147022FBF6A01A0
:103C20007B01EE24FF248C0120E030E0C016D10699
:103C3000E206F30610F4415051099A01281B390B92
:103C4000C9011F910F91FF90EF90DF90CF900895E1
:103C500078941F920F920FB60F9211248F939F9317
:103C6000AF93BF938091440290914502A091460288
:103C7000B09147020196A11DB11D8093440290931B
:103C80004502A0934602B0934702BF91AF919F9126
:103C90008F910F900FBE0F901F90189581E0809329
:103CA000E00080E28093D8001092C9008FE19EE48A
:103CB0000197F1F700C0000087E090EBDC018093F2
:103CC000570290935802A0935902B0935A029CE075
:103CD00088E10FB6F894A895809360000FBE90938A
:103CE0006000FFCF0E94A61C811102C00E94201D0F
:103CF0000E94B11C809326020E94B91C90E0909310
:103D00004902809348020E94B51C682F70E080E051
:103D100090E00C94E41980912B0280FF0BC060911D
:103D20003A0185E0689FB0011124759567957595F6
:103D300067952BC081FF09C060913A0185E0689FBB
:103D4000B00111247595679520C082FF07C060916E
:103D50003A0185E0689FB001112417C090912A02B2
:103D60009923D1F060913901961788F720913A0193
:103D700085E0289F90011124929FA001939F500DF0
:103D8000112470E0CA010E94252E6038710540F4AC
:103D90006115710539F002C065E070E0862F089565
:103DA0008FE7089581E0089580912B0280FF08C07D
:103DB0006091380170E0759567957595679521C09C
:103DC00081FF06C06091380170E07595679519C054
:103DD00082FF04C06091380170E010C090912A0207
:103DE0009923C1F0609137019617A0F780913801AF
:103DF000899FC001112470E00E94252E6038710552
:103E000028F46115710521F0862F08958FE7089534
:103E100081E0089561E070E0F4CF803F21F40E94DA
:103E20008B1E819504C0813F29F40E948B1E8093D4
:103E30002F020895823F21F40E948B1E819504C0B9
:103E4000833F29F40E948B1E80932E020895893FA0
:103E500019F40E94D41E05C08A3F31F40E94D41E7A
:103E600081958093300208958B3F21F40E94D41EE7
:103E7000819504C08C3F29F40E94D41E80933102A6
:103E80000895843F21F480912D02816017C0853F01
:103E900021F480912D02826011C0863F21F480912F
:103EA0002D0284600BC0873F21F480912D02886031
:103EB00005C0883F31F480912D02806180932D02EE
:103EC00008958D3F21F480912B0281600BC08E3FBD
:103ED00021F480912B02826005C08F3F29F48091EC
:103EE0002B02846080932B020895803F39F48091E7
:103EF0002F0287FF6CC010922F0269C0813F29F406
:103F000080912F021816BCF362C090912E02823F5E
:103F100029F497FF5CC010922E0259C0833F19F418
:103F20001916CCF354C0893F41F480913002181621
:103F30000CF04DC0109230024AC08A3F29F48091A3
:103F4000300287FF44C0F6CF8B3F39F480913102B5
:103F500087FF3DC0109231023AC08C3F29F4809116
:103F600031021816BCF333C0843F21F480912D0236
:103F70008E7F17C0853F21F480912D028D7F11C067
:103F8000863F21F480912D028B7F0BC0873F21F467
:103F900080912D02877F05C0883F31F480912D02EA
:103FA0008F7E80932D0213C08D3F21F480912B02D0
:103FB0008E7F0BC08E3F21F480912B028D7F05C038
:103FC0008F3F29F480912B028B7F80932B0280916D
:103FD0002E0281110EC080912F0281110AC08091A2
:103FE0003002811106C080913102811102C010920D
:103FF0002A0208958091260283FF7EC081EB93E020
:104000000E94260780912D021F928F938CEA93E0E5
:104010009F938F930E94BF078AEA93E00E9426072E
:1040200080912E02282F082E000C330B3F938F9384
:1040300087EA93E09F938F930E94BF0785EA93E0FE
:104040000E94260780912F02282F082E000C330B88
:104050003F938F9382EA93E09F938F930E94BF07D1
:1040600080EA93E00E94260780913002282F082ED4
:10407000000C330B3F938F938DE993E09F938F93C5
:104080000E94BF078BE993E00E94260780913102CE
:10409000282F082E000C330B3F938F9388E993E071
:1040A0009F938F930E94BF0785E993E00E942607A4
:1040B00080912A021F928F9382E993E09F938F93BE
:1040C0000E94BF0780E993E00E94260780912B029F
:1040D0001F928F938DE893E09F938F930E94BF0769
:1040E0008AE893E00E9426078DB79EB74C960FB6DC
:1040F000F8949EBF0FBE8DBF8CE292E00E942C1000
:104100000E94E61D909329028093280208951F9330
:10411000CF93DF9380912802909129020E94FE1D87
:10412000AC0190912A02992321F020913B0130E0CB
:1041300006C020913C018AE0289F9001112442177B
:10414000530708F47BC080912E02C0912F02D091BA
:10415000300210913102811107C0C1116BC0D11121
:1041600069C0111167C06AC09F3F19F09F5F9093AB
:104170002A02181624F40E948B1E80932E0280912E
:104180002E0287FF05C00E948B1E819580932E0210
:104190001C1624F40E948B1E80932F0280912F0204
:1041A00087FF05C00E948B1E819580932F0230915E
:1041B0002E023323E1F020912F022223C1F045EBA0
:1041C0003403C0011124892F990F990B009709F42A
:1041D00081E080932E0235EB2303C0011124892F47
:1041E000990F990B009709F481E080932F021D1617
:1041F00024F40E94D41E809330028091300287FF05
:1042000005C00E94D41E819580933002111624F4BB
:104210000E94D41E809331028091310287FF05C035
:104220000E94D41E819580933102DF91CF911F911E
:104230000C94FA1F9F3F09F099CFA1CFDF91CF9146
:104240001F910895ECE2F2E086E0DF011D928A956D
:10425000E9F710922A0210922B02089584ED95E05E
:104260000E9426071F9281E08F931F9285E08F9313
:1042700086E895E09F938F930E94BF070F900F9061
:104280000F900F900F900F9008958330E9F128F46C
:10429000813061F0823009F10895853009F462C0FF
:1042A00008F449C0863009F474C0089580913C0137
:1042B000262F30E0280F311D2F3F310524F4680FE1
:1042C00060933C0103C08FEF80933C0180913C01DF
:1042D0001F928F938FEB94E072C080913B01262F49
:1042E00030E0280F311D2F3F310524F4680F609313
:1042F0003B0103C08FEF80933B0180913B011F92F4
:104300008F938DEA94E05BC080913A01262F30E0D4
:10431000280F311D2F3F310524F4680F60933A01B7
:1043200003C08FEF80933A0180913A011F928F93DF
:104330008AE994E044C080913901262F30E0280FAB
:10434000311D2F3F310524F4680F6093390103C0FC
:104350008FEF80933901809139011F928F9385E807
:1043600094E02DC080913801262F30E0280F311DB8
:104370002F3F310524F4680F6093380103C08FEF9D
:1043800080933801809138011F928F938CE694E0DE
:1043900016C080913701262F30E0280F311D2F3FA6
:1043A000310524F4680F6093370103C08FEF8093C9
:1043B0003701809137011F928F9381E594E09F939D
:1043C0008F930E94BF070F900F900F900F9008954A
:1043D000833081F128F4813059F08230D1F0089592
:1043E000853009F449C0B8F1863009F456C0089503
:1043F00080913C01681720F4861B80933C0102C029
:1044000010923C0180913C011F928F9382E494E0D2
:1044100054C080913B01681720F4861B80933B01B8
:1044200002C010923B0180913B011F928F9380E369
:1044300094E043C080913A01681720F4861B809372
:104440003A0102C010923A0180913A011F928F9373
:104450008DE194E032C080913901681720F4861B09
:104460008093390102C010923901809139011F9265
:104470008F9388E094E021C080913801681720F480
:10448000861B8093380102C0109238018091380158
:104490001F928F938FEE93E010C0809137016817C1
:1044A00020F4861B8093370102C01092370180915F
:1044B00037011F928F9384ED93E09F938F930E9417
:1044C000BF070F900F900F900F900895CF93C82FB4
:1044D0001F928F9389ED96E09F938F930E94BF0761
:1044E00081E090E0A0E0B0E0BC01CD0104C0660F27
:1044F000771F881F991FCA95D2F70E94E4190F9061
:104500000F900F900F90CF910C940916CF938B3191
:1045100009F4D1C108F067C18B3009F48AC108F0F1
:104520003DC1863009F488C120F4853009F496C174
:1045300044C2873009F4A4C1883009F03EC285EF37
:104540009BE00E94260786E49BE00E9426070E94CB
:10455000B51C1F928F9383E49BE09F938F930E94DF
:10456000BF0781E49BE00E9426070E94B11CC82F70
:104570008EE29BE00E9426071F92CF9389E29BE088
:104580009F938F930E94BF0787E29BE00E942607BC
:104590008DE19BE00E9426078C2F81701F928F93E4
:1045A0008AE19BE09F938F930E94BF0788E19BE085
:1045B0000E9426078EE09BE00E942607C1FB882709
:1045C00080F91F928F938BE09BE09F938F930E94C3
:1045D000BF0789E09BE00E9426078DEF9AE00E94CA
:1045E0002607C2FB882780F91F928F938AEF9AE0F3
:1045F0009F938F930E94BF0788EF9AE00E9426073F
:104600008FEE9AE00E942607C3FBCC27C0F91F92C9
:10461000CF938CEE9AE09F938F930E94BF078AEE10
:104620009AE00E9426070E94B91CC82F86ED9AE0E6
:104630000E9426071F92CF9381ED9AE09F938F935C
:104640000E94BF078FEC9AE00E94260786EB9AE053
:104650000E9426078C2F81701F928F9383EB9AE024
:104660009F938F930E94BF078DB79EB780960FB61A
:10467000F8949EBF0FBE8DBF81EB9AE00E94260783
:104680008AE99AE00E942607C1FB882780F91F92D9
:104690008F9387E99AE09F938F930E94BF0785E9E4
:1046A0009AE00E94260783E89AE00E942607C2FB50
:1046B000882780F91F928F9380E89AE09F938F93C9
:1046C0000E94BF078EE79AE00E9426078CE69AE0D8
:1046D0000E942607C3FB882780F91F928F9389E6E3
:1046E0009AE09F938F930E94BF0787E69AE00E940B
:1046F00026078DE59AE00E942607C4FB882780F9EB
:104700001F928F938AE59AE09F938F930E94BF0731
:1047100088E59AE00E94260786E49AE00E94260730
:10472000C5FB882780F91F928F9383E49AE09F93BB
:104730008F930E94BF0781E49AE00E94260785E2DA
:104740009AE00E942607C6FB882780F91F928F9364
:1047500082E29AE09F938F930E94BF0780E29AE0E3
:104760000E94260788E19AE00E942607C7FBCC2713
:10477000C0F91F92CF9385E19AE09F938F930E9497
:10478000BF0783E19AE00E9426078DB79EB74C963B
:104790000FB6F8949EBF0FBE8DBF49C0803109F49B
:1047A000B4C020F48E3009F49AC007C1863109F4F0
:1047B000C7C0893109F001C18AE398E00E94260749
:1047C00088E198E00E94260786EE97E00E9426077F
:1047D0008BEA97E00E94260785E797E00E9426076C
:1047E00087E497E08FC08A32E1F060F4873209F401
:1047F000E0C028F48E3108F4E0C08D51DBC089326E
:1048000069F1DBC0833448F48A3308F0D0C08533C3
:1048100009F4CFC0883369F0D0C0833409F4C9C02B
:10482000CCC084EE9BE00E9426070E94201DC1E0C0
:10483000C9C080E798E066C080912602817F8E7FA4
:104840008093260289E498E00E94260780EE9BE090
:104850000E94260781E080933302E9CF0E94091667
:1048600084EC9BE00E9426079FEF23ED80E39150AC
:1048700020408040E1F700C000000E944E1ED7CFCC
:1048800080912602C82FC095C170C0FB80F980932B
:104890002602CC2329F088EB9BE00E94260792C0D9
:1048A0008BEA9BE00E94260780912602897F877F02
:1048B00080932602BCCF9091260291FBCC27C0F9B1
:1048C00081E0C827892FC0FB81F980932602CC2381
:1048D00019F08EE99BE029C080E99BE013C090911C
:1048E000260292FBCC27C0F981E0C827892FC0FBA4
:1048F00082F980932602CC2319F081E89BE015C051
:1049000081E79BE00E94260792CF9091260293FBBD
:10491000CC27C0F981E0C827892FC0FB83F9809399
:104920002602CC2351F085E69BE00E942607809169
:10493000260281608093260245C088E59BE0E2CF95
:1049400089E397E00E9426070E94D70F1F928F935A
:104950008FE197E09F938F930E94BF07809147015B
:104960001F928F9388E097E09F938F930E94BF07D9
:10497000809140021F928F9385EF96E09F938F93D3
:104980000E94BF070E94F21D9F938F937F936F93A6
:104990008EED96E09F938F930E94BF078DB79EB7D1
:1049A00042960FB6F8949EBF0FBE8DBF40CF89537D
:1049B00001C080E00E9466223ACF86E59BE00E941B
:1049C0002607C0E08C2FCF91089580E0089580E005
:1049D00008958E518A3030F4E82FF0E0E45AFE4F0B
:1049E0008081089580E00895CF93C82F809133028D
:1049F000813059F020F0823009F445C039C10E945D
:104A0000BE1B823209F036C104C00E94BE1B823236
:104A100061F48C2F0E94E524811104C08C2F0E9428
:104A200086222FC081E090E02CC08C2F0E94E724CA
:104A3000811126C0C431E1F070F4CB3081F0C03177
:104A4000D1F40E942E2181ED96E00E94260782E09B
:104A50008093330215C0C93259F0C83361F489E438
:104A600098E00E94260785ED96E00E94260708C080
:104A70001092330201C18FEC96E00E942607FCC021
:104A800081E08170FBC0C43228F5CE3108F0C1C08E
:104A9000CB30A1F1D0F4C73009F0D0C08EE18093C3
:104AA0003C0182E380933B018AE080933A0184E1F8
:104AB0008093390188E08093380188E28093370140
:104AC00085E795E00E942607BCC0C33149F1C43197
:104AD000C1F0B4C0CB3409F4A6C028F4C93289F0BF
:104AE000C83361F0ABC0C13509F49BC0C23509F4CD
:104AF00096C0CE3409F0A2C06AE09BC00E942E216D
:104B0000A0C080913202882319F01092320299C01D
:104B100082E895E00E94260781E080933302AEC0D0
:104B20008CE595E00E9426078AE495E00E9426071E
:104B300080913C011F928F9387E495E09F938F9320
:104B40000E94BF0785E495E00E94260783E395E075
:104B50000E94260780913B011F928F9380E395E08E
:104B60009F938F930E94BF078EE295E00E942607D5
:104B70008FE195E00E94260780913A011F928F9362
:104B80008CE195E09F938F930E94BF078AE195E0A7
:104B90000E94260789E095E00E942607809139014E
:104BA0001F928F9386E095E09F938F930E94BF079B
:104BB00084E095E00E9426078FEE94E00E9426078D
:104BC000809138011F928F938CEE94E09F938F9386
:104BD0000E94BF078AEE94E00E94260783ED94E0CE
:104BE0000E942607809137011F928F9380ED94E0F9
:104BF0009F938F930E94BF078EEC94E00E9426073C
:104C00008DB79EB748960FB6F8949EBF0FBE8DBF66
:104C100018C08C2F0E94E9248093320212C061E0F8
:104C200003C061E006C06AE0809132020E94452123
:104C300008C0809132020E94E82103C083E795E01A
:104C400013C080913202882369F01F928F938DE602
:104C500095E09F938F930E94BF070F900F900F9046
:104C60000F9004C08AE695E00E94260781E006C006
:104C70001092330280E002C080E003CFCF9108950C
:104C800080913F0208959FB7F894109236029FBF1B
:104C900090914E02943009F057C09091E9009F70B6
:104CA0003091EC00232F217030FD20E8922B23E07F
:104CB0002093E9002091EB0020FF43C02091EE00FB
:104CC00027FF3FC020913402222321F02091E800E9
:104CD00025FF37C01092340226E03091E80035FD00
:104CE00015C030914E02343061F53091EB0035FD46
:104CF00028C0215021F481E08093340222C0EFE9E2
:104D0000FFE03197F1F700C00000E7CF8093F1009A
:104D10008091E80085FD0AC08091E80080FFFCCF0B
:104D20008091E8008E778093E80006C08FB7F894F2
:104D300021E0209336028FBF9F709093E90080E0BE
:104D400008959F709093E9008FEF08950F931F933C
:104D5000CF93DF9300D01F92CDB7DEB78C010E94B6
:104D60006129823011F0843021F584E089831B832E
:104D70000A8382E08093E9008FEF9091E8008150F0
:104D800095FD06C095ED9A95F1F700008111F5CFDC
:104D90008091E80085FF0DC040E050E063E070E0E6
:104DA000CE0101960E947E298091E8008E77809343
:104DB000E8000F900F900F90DF91CF911F910F910E
:104DC0000895CF93DF9300D01F92CDB7DEB7209127
:104DD0004E02243031F523E02983805891099B83CA
:104DE0008A8382E08093E9008FEF9091E800815000
:104DF00095FD06C095ED9A95F1F700008111F5CF6C
:104E00008091E80085FF0DC040E050E063E070E075
:104E1000CE0101960E947E298091E8008E778093D2
:104E2000E8000F900F900F90DF91CF910895CF93EE
:104E3000DF93EC010E946129823011F08430F9F493
:104E400082E08093E9009FEF8091E800915085FD1A
:104E500006C085ED8A95F1F700009111F5CF80919C
:104E6000E80085FF0CC040E050E066E070E0CE0155
:104E70000E947E298091E8008E778093E800DF9180
:104E8000CF910895CF93DF93EC010E946129823086
:104E900011F0843039F581E08093E9008FEF909133
:104EA000E800815095FD06C095ED9A95F1F7000058
:104EB0008111F5CF8091E80085FF14C040E050E0FB
:104EC00068E070E0CE010E947E298091E8008E7734
:104ED0008093E80088E0FE01A7E3B2E001900D9224
:104EE0008A95E1F7DF91CF91089585E29CE00E94D9
:104EF000260780914D02811109C00E94132B0E9448
:104F0000702B8091E20084608093E200089581E23A
:104F10009CE00E94260710924D0208958DE19CE0CE
:104F20000C94260789E19CE00C94260785E19CE01F
:104F30000E9426070C94AC1D209135022F5F822F12
:104F400062E30E94192E992319F0209335020895E7
:104F50001092350280913602882371F180914E02C1
:104F6000843041F58091E9008F702091EC00922F00
:104F7000917020FD90E8892B93E09093E900909147
:104F8000EB0090FF14C09091EE0097FF10C090913D
:104F9000E80095FF03C01092F100F9CF9091E8006E
:104FA00090FF05C09091E8009E779093E8008F7085
:104FB0008093E90010923602089542E061EC81E0AE
:104FC0000E948D2A42E261EC82E00E948D2A42E238
:104FD00061EC83E00C948D2A80915002833009F4B7
:104FE00060C030F4813071F0823009F499C00895C6
:104FF0008A3009F485C08B3009F46BC0893009F020
:10500000A7C020C080914F02813A09F0A1C08091D1
:10501000E800877F8093E8008091530290915402CA
:10502000892B21F468E087E392E003C060E080E030
:1050300090E070E00E94C9298091E8008B7780930E
:10504000E800089580914F02813209F081C080917B
:10505000530290915402029708F07AC08091E800C0
:10506000877F8093E8008091E80082FD05C08091F1
:105070004E028111F8CF6CC02091F3008091F200B4
:1050800090E0922B029729F48091F1008B7F813080
:1050900021F48091F10080933F028091E8008B77AA
:1050A00053C080914F02813A09F052C0809153025F
:1050B00090915402892B09F04BC08091E800877FC2
:1050C0008093E8008091E80080FFFCCF8091470149
:1050D00036C080914F028132D9F580915302909170
:1050E0005402892BA9F58091E800877F8093E8001E
:1050F0000E94C22A80915102809347010C940916A4
:1051000080914F02813221F58091E800877F809362
:10511000E8000E94C22A80915202809340020895C2
:1051200080914F02813AA1F48091E800877F8093BB
:10513000E8008091E80080FFFCCF809140028093DE
:10514000F1008091E8008E778093E8000C94C22AE9
:10515000089584B7877F84BF0FB6F894A89580918F
:105160006000886180936000109260000FBE80E84C
:1051700080936100109261000E9474100E94132BB2
:105180000E94702B8091E20084608093E20083E4AF
:1051900096E20E94711C78940E94FE2D0E947C1061
:1051A0008DE391E00E94D20F84E09CE00E942607EC
:1051B00080914E02853089F480E09CE00E942607B1
:1051C0000E94621D80914C02882391F30E94941DDD
:1051D000882371F30E946829EBCF0E94AC10E8CFBE
:1051E0000C94F228292F332723303105C9F064F4B9
:1051F0002130310581F02230310509F049C08BE5BD
:1052000090E02DE43CE048C02132310521F122320A
:10521000310571F13DC082E190E028EA3CE03CC0FC
:1052200099278130910571F02CF4892B89F5E9E4F7
:10523000FCE00DC08230910541F0039749F5E9E2A9
:10524000FCE005C0EDE3FCE002C0EFE2FCE084918D
:1052500090E09F0121C063307105D0F4660F771F85
:10526000FB01E159FE4F2081318189E090E014C0BB
:105270006330710568F4FB01EE0FFF1FE759FE4F25
:1052800020813181FB01EA59FE4F808190E004C00A
:1052900080E090E020E030E0FA013183208308953F
:1052A0000895CF93C82F0E945029C0934102CF91F7
:1052B000089580914E02843011F081E0089582E0DB
:1052C000089580914102811102C00C9459290895DA
:1052D00080E189BD82E189BD09B400FEFDCF8091E6
:1052E000D8008F7D8093D8008091E0008260809309
:1052F000E0008091E00081FDFCCF0895CF92DF9225
:10530000EF92FF920F931F93CF93DF93EC018B01EA
:105310006A010E94E12A811133C0C114D10439F01D
:10532000F60180819181081B190BC80FD91FE12C50
:10533000F12C0115110519F18091E80085FD16C0C9
:105340008091E8008E778093E800C114D10449F081
:10535000F60180819181E80EF91EF182E08285E0FC
:105360000FC00E94E12A882321F30AC0899180930B
:10537000F10001501109FFEFEF1AFF0ADACF80E0C8
:10538000DF91CF911F910F91FF90EF90DF90CF9021
:10539000089520915502309156022617370748F09C
:1053A0006115710539F42091E8002E772093E8000B
:1053B00001C0B90140E061157105A9F120914E02CB
:1053C000222309F443C0253009F442C02091E800AB
:1053D00023FD40C02091E80022FD32C02091E8006A
:1053E00020FFE9CF4091F3002091F20030E0342B10
:1053F000FC01CF016115710559F02830310540F4E9
:1054000081918093F100615071092F5F3F4FF1CF7F
:1054100041E02830310509F040E02091E8002E7786
:105420002093E800C8CF4111C9CF0AC080914E0235
:10543000882361F0853061F08091E80083FD0AC027
:105440008091E80082FFF2CF80E0089582E0089525
:1054500083E0089581E0089520915502309156022D
:105460002617370748F06115710539F42091E800D7
:105470002E772093E80001C0B901FC0120E06115FE
:10548000710591F180914E02882309F440C0853066
:1054900009F43FC08091E80083FD3DC08091E800A1
:1054A00082FD2FC08091E80080FFE9CF2091F300BA
:1054B0008091F20090E0922B6115710559F08830CF
:1054C000910540F424912093F100319661507109C7
:1054D0000196F2CF21E0089709F020E08091E800E2
:1054E0008E778093E800CBCF2111CCCF0AC080917A
:1054F0004E02882361F0853061F08091E80083FDE1
:105500000AC08091E80082FFF2CF80E0089582E037
:10551000089583E0089581E00895982F973058F515
:105520009093E900981739F07091EC002091ED000C
:105530005091F00003C0242F762F50E021FF19C0B6
:105540003091EB003E7F3093EB003091ED003D7FDA
:105550003093ED003091EB0031603093EB007093AD
:10556000EC002093ED005093F0002091EE0027FF17
:1055700007C09F5FD3CF8F708093E90081E00895CB
:1055800080E0089580914F0287FF11C08091E8006C
:1055900082FD05C080914E028111F8CF11C080912B
:1055A000E8008B770BC080914E02882349F08091F0
:1055B000E80080FFF8CF8091E8008E778093E800C4
:1055C00008952091E4003091E50095E64091EC00CB
:1055D000842F817040FF22C08091E80080FD1CC0B4
:1055E00080914E02882391F0853091F08091EB00FC
:1055F00085FD10C04091E4005091E500421753072B
:1056000029F39A01915011F784E0089582E00895FA
:1056100083E0089581E0089580E008954091E800D6
:1056200042FFDECF08950E94812B0E94892BE0EE7D
:10563000F0E0808181608083E8EDF0E080818F7709
:10564000808319BCA7EDB0E08C918E7F8C93808114
:105650008F7E808310924D0208950F931F93CF93F6
:10566000DF930E94812B0E94892BC8EDD0E08881B6
:105670008F77888388818068888388818F7D8883FD
:1056800019BC10924E0210924A0210924C021092D3
:105690004B0200EE10E0F80180818B7F80838881CF
:1056A0008160888342E060E080E00E948D2AE1EE24
:1056B000F0E080818E7F8083E2EEF0E08081816087
:1056C0008083808188608083F80180818E7F8083E1
:1056D000888180618883DF91CF911F910F91089518
:1056E000E8EDF0E080818F7E8083E7EDF0E080815F
:1056F0008160808384E082BF81E080934D020C94BE
:105700002D2BE8EDF0E080818E7F80831092E20007
:1057100008951092DA001092E10008951F920F92FE
:105720000FB60F9211242F933F934F935F936F9374
:105730007F938F939F93AF93BF93EF93FF9380914A
:10574000E10082FF0BC08091E20082FF07C08091E0
:10575000E1008B7F8093E1000E949C278091DA001A
:1057600080FF1FC08091D80080FF1BC08091DA00AD
:105770008E7F8093DA008091D90080FF0DC080E198
:1057800089BD82E189BD09B400FEFDCF81E080932F
:105790004E020E94752705C019BC10924E020E944D
:1057A00087278091E10080FF19C08091E20080FF8F
:1057B00015C08091E2008E7F8093E2008091E2002C
:1057C00080618093E2008091D80080628093D8004D
:1057D00019BC85E080934E020E9492278091E100DF
:1057E00084FF30C08091E20084FF2CC080E189BD3D
:1057F00082E189BD09B400FEFDCF8091D8008F7D84
:105800008093D8008091E1008F7E8093E1008091A9
:10581000E2008F7E8093E2008091E20081608093BD
:10582000E20080914A02882311F084E007C0809151
:10583000E30087FD02C081E001C083E080934E0257
:105840000E9496278091E10083FF29C08091E200A9
:1058500083FF25C08091E100877F8093E10082E093
:1058600080934E0210924A028091E1008E7F8093D5
:10587000E1008091E2008E7F8093E2008091E2005F
:1058800080618093E20042E060E080E00E948D2A27
:105890008091F00088608093F0000E948E27FF9135
:1058A000EF91BF91AF919F918F917F916F915F9198
:1058B0004F913F912F910F900FBE0F901F90189511
:1058C0001F920F920FB60F9211242F933F934F9375
:1058D0005F936F937F938F939F93AF93BF93CF9378
:1058E000DF93EF93FF93C091E900CF708091EC00BC
:1058F000D82FD17080FDD0E81092E9008091F0009F
:10590000877F8093F00078940E94A42C1092E90085
:105910008091F00088608093F000CD2BCF70C09311
:10592000E900FF91EF91DF91CF91BF91AF919F91EE
:105930008F917F916F915F914F913F912F910F9038
:105940000FBE0F901F9018951F93CF93DF93CDB785
:10595000DEB7AA970FB6F894DEBF0FBECDBFEFE457
:10596000F2E088E08E0F9091F10091938E13FBCFBF
:105970000E94EC278091E80083FF28C180914F02AC
:1059800090915002492F50E04A30510508F01EC155
:10599000FA01E556FF4F0C94392E803821F08238F9
:1059A00009F014C108C080914B0290914C029923D8
:1059B00089F082600FC0809153028F70873008F0A9
:1059C00005C18093E9008091EB0085FB882780F971
:1059D0001092E9009091E800977F9093E8008093FF
:1059E000F1001092F100D0C0282F2D7F09F0EEC0F9
:1059F000882319F0823061F0E9C080915102813032
:105A000009F0E4C0933009F080E080934C022EC08E
:105A10008091510281112AC0809153028F702FEF23
:105A2000280F263008F0D2C08093E9002091EB00C7
:105A300020FF1CC0933021F48091EB00806214C0E1
:105A40009091EB0090619093EB0021E030E0A90190
:105A500002C0440F551F8A95E2F74093EA00109266
:105A6000EA008091EB0088608093EB001092E900DF
:105A70008091E800877F8093E8000E94C22AA6C038
:105A80008111A4C0109151021F778091E3008078AA
:105A9000812B8093E3008091E800877F8093E8006A
:105AA0000E94C22A8091E80080FFFCCF8091E30031
:105AB00080688093E300111102C082E001C083E09E
:105AC00080934E0283C08058823008F07FC080915E
:105AD0005102909152028C3D53E0950779F583E095
:105AE0008A838AE289834FB7F894DE01139620E017
:105AF0003EE051E2E32FF0E050935700E49120FFA5
:105B000003C0E295EF703F5FEF708E2F90E0EA30B8
:105B100010F0C79601C0C0968D939D932F5F2431DE
:105B200049F74FBF8091E800877F8093E8006AE2E1
:105B300070E0CE0101960E94C92915C06091530200
:105B400070915402AE014F5F5F4F0E94F028BC017C
:105B5000892BE1F19091E800977F9093E80089818B
:105B60009A810E942C2A8091E8008B778093E8002C
:105B70002DC0803859F58091E800877F8093E80038
:105B800080914A028093F1008091E8008E7773CF74
:105B900081111CC0909151029230C0F48091E800B4
:105BA000877F8093E80090934A020E94C22A8091E6
:105BB0004A02811106C08091E30087FD02C081E0A6
:105BC00001C084E080934E020E94DD278091E800AE
:105BD00083FF0AC08091E800877F8093E80080916E
:105BE000EB0080628093EB00AA960FB6F894DEBFBC
:105BF0000FBECDBFDF91CF911F910895CF938091BC
:105C00004E028823A1F0C091E900CF709091EC0082
:105C1000892F817090FD80E8C82B1092E900809157
:105C2000E80083FD0E94A42CCF70C093E900CF91BF
:105C30000895991B79E004C0991F961708F0961BE8
:105C4000881F7A95C9F78095089597FB072E16F45B
:105C5000009407D077FD09D00E943F2E07FC05D0A5
:105C60003EF4909581959F4F0895709561957F4F73
:105C70000895EE0FFF1F0590F491E02D0994AA1BE3
:105C8000BB1B51E107C0AA1FBB1FA617B70710F027
:105C9000A61BB70B881F991F5A95A9F78095909559
:105CA000BC01CD010895F999FECF92BD81BDF89A4E
:105CB000992780B50895A8E1B0E042E050E00C9447
:105CC000872E262FF999FECF92BD81BDF89A0197B4
:105CD00000B4021639F01FBA20BD0FB6F894FA9A34
:105CE000F99A0FBE08950396272F0E94622E0E94F4
:105CF000612E252F0E94622E242F0C94622E019675
:105D0000272F0E94622E0C94612EDC01CB01FC0136
:105D1000F999FECF06C0F2BDE1BDF89A319600B404
:0E5D20000D9241505040B8F70895F894FFCF0F
:105D2E00BF0DD00DE00D00000000000000000000CF
:105D3E00000000003001BF0DD00DE00D000000008E
:105D4E00000000000000000000002C01E600E7004B
:105D5E00E200E300FF1B022808140A321E4026420E
:105D6E00271727E126A62601F0F1C667663694317D
:105D7E003037353497963390919293950102030400
:105D8E00050607080900408522610DDC0CBA0C5F80
:065D9E000C780C910C00D2
:00000001FF
